:100000000C94DE000C9406010C9406010C94D10FA4
:100010000C94D10F0C94D10F0C9406010C94060192
:100020000C9406010C9406010C9406010C94060134
:100030000C9406010C9406010C9406010C94060124
:100040000C942F0F0C9406010C949F0F0C94790FB5
:100050000C9406010C9406010C9406010C94060104
:100060000C9449100C9406010000000023002600A7
:10007000290000000000240027002A004F4B204BDD
:1000800020004F4B204B00455252004F4B20760032
:1000900045525200B4B4B4B4B4B4B4B4B4B4B4B407
:1000A000B4B4B4B4B4B4B4B4B4B4B4B4B4B4B4B410
:1000B000B4B4B4B400000000000000000000000070
:1000C0000000000000000000000000000000000030
:1000D000000000005A5A5A5A5A5A5A5A5A5A5A5AE8
:1000E0005A5A5A5A5A5A5A5A5A5A5A5A5A5A5A5A70
:1000F0005A5A5A5AC409C409C409C409C409C409CA
:10010000C409C409C409C409C409C409C409C40987
:10011000C409C409C409C409C409C409C409C40977
:10012000C409C409C409C409C409C409C409C40967
:10013000C409C409F401F401F401F401F401F40167
:10014000F401F401F401F401F401F401F401F40107
:10015000F401F401F401F401F401F401F401F401F7
:10016000F401F401F401F401F401F401F401F401E7
:10017000F401F40100000000250028002B00040415
:10018000040404040404020202020202030303033F
:10019000030301020408102040800102040810201B
:1001A0000102040810200000000800020100000302
:1001B00004070000000000000000861211241FBE8A
:1001C000CFEFD8E0DEBFCDBF11E0A0E0B1E0E0EAC4
:1001D000F3E302C005900D92A234B107D9F725E0F0
:1001E000A2E4B1E001C01D92A43FB207E1F710E024
:1001F000CEEDD0E004C02197FE010E948918CD3DCC
:10020000D107C9F70E94D7120C94CE190C940000A4
:100210000895089590E0FC01EA55FE4F2491FC01F9
:10022000EE56FE4F3491FC01E258FE4FE491EE236E
:10023000C9F0222339F0233001F1A8F4213019F15B
:10024000223029F1F0E0EE0FFF1FEC58FE4FA59190
:10025000B4918FB7F894EC91611126C030953E238C
:100260003C938FBF08952730A9F02830C9F024307F
:1002700049F7809180008F7D03C0809180008F7747
:1002800080938000DFCF84B58F7784BDDBCF84B5CA
:100290008F7DFBCF8091B0008F778093B000D2CF5D
:1002A0008091B0008F7DF9CF3E2BDACF3FB7F89425
:1002B0008091BB049091BC04A091BD04B091BE0498
:1002C00026B5A89B05C02F3F19F00196A11DB11DB1
:1002D0003FBFBA2FA92F982F8827BC01CD01620FED
:1002E000711D811D911D42E0660F771F881F991FA8
:1002F0004A95D1F708958F929F92AF92BF92CF9275
:10030000DF92EF92FF924B015C010E9456016B015C
:100310007C010E9456016C197D098E099F09683E77
:10032000734081059105A8F321E0821A9108A10884
:10033000B10888EEC80E83E0D81EE11CF11C8114C0
:100340009104A104B10429F7FF90EF90DF90CF90C2
:10035000BF90AF909F908F900895EF92FF920F9370
:100360001F93CF93DF938C017B01D0E0C0E0F701B6
:10037000EC0FFD1F6491662361F0D801ED91FC91B3
:100380000190F081E02DC8010995892B11F021968B
:10039000EECFCE01DF91CF911F910F91FF90EF90A3
:1003A0000895AF92BF92CF92DF92EF92FF920F9398
:1003B0001F93CF93DF936C017B018B01040F151FFB
:1003C000EB015E01AE18BF08C017D10759F0699163
:1003D000D601ED91FC910190F081E02DC6010995C7
:1003E000892B79F7C501DF91CF911F910F91FF9074
:1003F000EF90DF90CF90BF90AF900895FC01538DA8
:10040000448D252F30E0842F90E0821B930B5417EE
:1004100010F0CF96089501970895FC01918D828D7B
:10042000981761F0A28DAE0FBF2FB11D5D968C9114
:10043000928D9F5F9F73928F90E008958FEF9FEF53
:100440000895FC01918D828D981731F0828DE80F0F
:10045000F11D858D90E008958FEF9FEF0895FC01C9
:10046000918D228D892F90E0805C9F4F821B910996
:100470008F739927089585E395E00E942F0221E06C
:10048000892B09F420E0822F089580E090E0892BE9
:1004900029F00E943B0281110C9400000895FC0198
:1004A000A48DA80FB92FB11DA35ABF4F2C91848DD5
:1004B00090E001968F739927848FA689B7892C9332
:1004C000A089B1898C91837080648C93938D848D85
:1004D000981306C00288F389E02D80818F7D808388
:1004E0000895EF92FF920F931F93CF93DF93EC0148
:1004F00081E0888F9B8D8C8D98131AC0E889F989CB
:10050000808185FF15C09FB7F894EE89FF896083CD
:10051000E889F98980818370806480839FBF81E04E
:1005200090E0DF91CF911F910F91FF90EF90089590
:10053000F62E0B8D10E00F5F1F4F0F731127E02E6B
:100540008C8D8E110CC00FB607FCFACFE889F989A3
:10055000808185FFF5CFCE010E944F02F1CFEB8D58
:10056000EC0FFD2FF11DE35AFF4FF0829FB7F89477
:100570000B8FEA89FB8980818062CFCFCF93DF9395
:10058000EC01888D8823B9F0AA89BB89E889F989AB
:100590008C9185FD03C0808186FD0DC00FB607FCE0
:1005A000F7CF8C9185FFF2CF808185FFEDCFCE0113
:1005B0000E944F02E9CFDF91CF9108952091CC01A5
:1005C0003091CD012817390771F49091CB018091BA
:1005D000CA01981741F0E091CB01F0E0E657FE4FD9
:1005E000808190E008958FEF9FEF08950895EF9236
:1005F000FF920F931F93CF93DF93DC015C96ED90F6
:10060000FC905D97E114F10479F481E090E0139699
:100610009C938E93129790E080E0DF91CF911F9191
:100620000F91FF90EF9008955196ED91FC915297A4
:1006300050968C915097982F90950FB75E962C916D
:100640005E97122F127021FD6095F894208111237E
:1006500019F1282B2083E7012197F1F728E0462F95
:1006600050E0308160FF1AC0382B3083E7012197BA
:10067000F1F7BA0175956795215089F7112381F03B
:100680008081892380830FBF5C968D919C91019717
:10069000F1F781E090E0C1CF2923DCCF3923E5CF0A
:1006A0009081892BEFCF2091CC013091CD0128177B
:1006B000390761F48091CA012091CB0190E0805C00
:1006C0009F4F821B91098F739927089590E080E0D6
:1006D00008952091CC013091CD0128173907B9F444
:1006E0009091CB018091CA01981789F0E091CB01DC
:1006F000F0E0E657FE4F80812091CB0130E02F5F84
:100700003F4F2F7333272093CB0190E008958FEF55
:100710009FEF0895E091CC01F091CD01E817F90722
:1007200069F4A389B4899C918589809589238C93E8
:100730001092CD011092CC0181E0089580E00895DF
:1007400020916701260F3327331F21323105ECF446
:1007500020910B05FC0190E080E0243069F082E0FC
:100760000895A09167012191AC01495B5E4FA40FF0
:10077000B52FB11D2C930196861798F380916701D0
:10078000680F6093670180E0089581E008951092FA
:100790000B0581E080930A051092E50461E082E197
:1007A0000E940A0161E083E10E940A01E9EBF0E0A6
:1007B00080818E7F808380818D7F808388E4809399
:1007C000B80085E48093BC0008951092C404109290
:1007D000C30410921205109234050E94C70388E0EA
:1007E00091E09093C2048093C10489E091E09093DA
:1007F000C0048093BF040895CF93DF9391E090935A
:1008000046018823B9F0C091B800D091BA00809118
:10081000BC008A7B8093BC0060E082E10E940A01F8
:1008200060E083E10E940A010E94C703D093BA00EE
:10083000C093B800DF91CF9108958F929F92AF92AD
:10084000BF92CF92DF92EF92FF920F931F93CF93BD
:10085000DF93D0913405D13208F0D7C0182FC09162
:1008600033050E9456016B017C0180910B058111BB
:100870006BC082E080930B0510930A058FEF809385
:10088000090510920805D0930705A3E1B5E0E7EE4E
:10089000F4E080E0D81391C01092E6048091E60461
:1008A000CC0FC82BC093E6048091E504813009F099
:1008B00088C01092E5040E9456016B017C01809172
:1008C000E6048093BB0080910D0590910E05A091E8
:1008D0000F05B0911005892B8A2B8B2BA1F00E945C
:1008E000560100910D0510910E0520910F053091D4
:1008F00010056C197D098E099F090617170728072F
:10090000390708F442C08091BC0083FDD8CF85EC44
:100910008093BC000E9456016B017C0180910B0505
:10092000823009F450C0809109058F3F09F46FC0EF
:1009300080910905803209F46CC0809109058033EB
:1009400009F469C084E026C080910D0590910E05E0
:10095000A0910F05B0911005892B8A2B8B2B09F4E0
:1009600084CF0E94560180900D0590900E05A090B6
:100970000F05B09010056C197D098E099F09861628
:100980009706A806B90608F070CF80910C050E9462
:10099000FC0385E0109212051092340510921105A7
:1009A000DF91CF911F910F91FF90EF90DF90CF904B
:1009B000BF90AF909F908F9008959D9191938F5F7E
:1009C00069CF85EEA5CF80910D0590910E05A09180
:1009D0000F05B0911005892B8A2B8B2B09F49ECF24
:1009E0000E94560100910D0510910E0520910F05F2
:1009F000309110056C197D098E099F09061717079C
:100A00002807390708F08ACFC0CF81E0C3CF80E044
:100A1000C1CF82E0BFCF83E0BDCF1F93CF93DF93E1
:100A2000EA01122FDC0111968D919C91DC01ED9170
:100A3000FC910280F381E02D0995C817D90729F4AC
:100A4000812F0E941D0491E0811190E0892FDF9198
:100A5000CF911F910895CF93DF93EC018B81882371
:100A6000A1F0888191E09093110580933305109255
:100A700012051092340581E00E941D0491E081115D
:100A800090E0892FDF91CF9108950E94E50381E0E6
:100A90008B83CE010E942B05982F8111E2CFF1CFDD
:100AA000E091C4048091C304E81730F4F0E0EB5304
:100AB000FB4F808190E008958FEF9FEF0895909114
:100AC000C4048091C3042FEF3FEF981748F4E92F37
:100AD000F0E0EB53FB4F208130E09F5F9093C40424
:100AE000C90108958091C3049091C404891B990B96
:100AF0000895CF92DF92EF92FF920F931F93CF93BF
:100B0000DF937C01CB018A0120911105222389F01A
:100B1000EB016B01C40ED51ECC15DD0569F06991A2
:100B2000D701ED91FC910190F081E02DC70109956D
:100B3000F3CF642F0E94A003C801DF91CF911F91D2
:100B40000F91FF90EF90DF90CF900895CF93DF93B8
:100B50001F92CDB7DEB76983209111052223F9F0EA
:100B600020913405203258F021E030E0FC0133833D
:100B7000228390E080E00F90DF91CF9108958091E3
:100B80001205E82FF0E0ED5EFA4F998190838F5FB8
:100B9000809312058093340581E090E0ECCF61E012
:100BA000CE0101960E94A003F7CF90E080E0089567
:100BB0008F929F92AF92BF92CF92DF92EF92FF926D
:100BC000CF93DF93653B710514F064EB70E0282F41
:100BD00030E0F901E852FD4F408150E077FF02C05C
:100BE00070E060E0461757070CF4AB01F901E854D8
:100BF000FD4FE081F0E04E175F070CF4FA016E2F15
:100C0000D901A858BC4FEC93C12CD12C7601C394C8
:100C100004C0CC0CDD1CEE1CFF1C8A95D2F7809022
:100C2000980390909903A0909A03B0909B03D701EA
:100C3000C60188219921AA21BB21892B8A2B8B2BC4
:100C4000E1F4220F331F220F331FE901C850DD4F9B
:100C500070E090E080E00E942417688379838A83A3
:100C60009B838C289D28AE28BF2880929803909261
:100C70009903A0929A03B0929B03809142019091B4
:100C80004301A0914401B09145018C299D29AE29D1
:100C9000BF298093420190934301A0934401B093F4
:100CA0004501DF91CF91FF90EF90DF90CF90BF9003
:100CB000AF909F908F90089590910201891758F5F9
:100CC000403991E059073CF19B0169327A4014F0B8
:100CD00028E23AE02039F1E03F0714F420E931E05E
:100CE00049329AE0590714F048E25AE024173507D0
:100CF00094F490E0880F991FFC01E25DFD4F318371
:100D00002083FC01E251FE4F5183408388589D4F60
:100D1000FC0111821082089590910201891768F4F4
:100D2000E82FF0E0E253FE4F9B01653B710514F0A4
:100D300024EB30E037FD20E02083089590910201FC
:100D4000891770F59B01653B710514F024EB30E0C9
:100D500037FF02C030E020E057FD23C0453B51057E
:100D60001CF5421753072CF4622F932F9A01462F3C
:100D7000592F90E0FC01E852FD4F2083FC01E8541C
:100D8000FD4F4083FC01E858FC4F808190E08217C2
:100D900093070CF4C901841795070CF4AC01408348
:100DA000089550E040E0DDCF44EB50E0E2CF909179
:100DB0000201891710F40C94D80508958F929F9220
:100DC000AF92BF92CF92DF92EF92FF92CF93DF93D9
:100DD000C82F6A017B0120E030E0A901CB01B601F8
:100DE0000E947E1687FD4AC020E030E044E353E4D1
:100DF000C701B6010E94D617181634F4C12CD12CA5
:100E000094E3E92E93E4F92E2C2F30E0220F331FC8
:100E1000F901E25DFD4FC081D18122513E4FF901C0
:100E2000608171816C1B7D0B90E080E00E94241733
:100E30004B015C0120E030E044E353E4C701B6011C
:100E40000E9483169B01AC01C501B4010E94DB170F
:100E500020E030E040E05FE30E9412160E94F516A9
:100E6000CE01860F971FDF91CF91FF90EF90DF901B
:100E7000CF90BF90AF909F908F900895C12CD12CB0
:100E80007601C2CFFC01808191818334924549F57E
:100E90004281538164817581368127818085932FBA
:100EA0009227A5EA9A279827942795279627E185E0
:100EB000E91317C09EEF930F9C3098F49EEF920FAA
:100EC0009C3078F4321769F08150823050F4405BE6
:100ED00054406109710981E041355D4B6140710504
:100EE00008F080E008951F93CF93DF9300D000D0E7
:100EF0001F92CDB7DEB7660F660F6A5F69831A82ED
:100F00001B824C835D83FC0183819481FC012481DD
:100F1000358125303105E0F0208111E01093110575
:100F200020933305109212051092340521E045E01C
:100F300050E0BE016F5F7F4F0E940D0581270F902B
:100F40000F900F900F900F90DF91CF911F91089508
:100F500081E0F5CF682FE82FF0E0EE0FFF1FE85893
:100F6000FD4F1182108240E050E187EE95E0603144
:100F700028F0605140E050E18EED95E00C9473074D
:100F80002F923F924F925F926F927F928F929F9299
:100F9000AF92BF92CF92DF92EF92FF920F931F9387
:100FA000CF93DF93DC0114962D913C911597232B61
:100FB00009F40FC14A01EC01888191E09093110579
:100FC00080933305109212051092340520E041E021
:100FD00050E0CD010E940D05F82E882309F4F9C0D8
:100FE000EE24E39485EC382ECC80DD8001E0C11442
:100FF000D10409F400E0A02EB12C28800E945601F3
:101000002B013C0180910B05811165C0102FE092EE
:101010000B0500930A05BFEFB09309051092080570
:101020008FEF800F80930705E092E6048091E6043D
:10103000220C282A2092E6048091E504813009F0F0
:101040008BC01092E5040E9456012B013C01809157
:10105000E6048093BB0080910D0590910E05A09150
:101060000F05B0911005892B8A2B8B2BA1F00E94C4
:10107000560120910D0530910E0540910F055091BC
:101080001005641975098609970926173707480757
:10109000590708F441C08091BC0083FDD8CF30923D
:1010A000BC000E9456012B013C0180910B05813050
:1010B00009F456C080910805801710F410910805B6
:1010C000E7EEF4E0A5ECB4E080E0811751F19191F6
:1010D0009D938F5FFACF80910D0590910E05A091A1
:1010E0000F05B0911005892B8A2B8B2B09F48ACF21
:1010F0000E94560120910D0530910E0540910F057B
:101100005091100564197509860997092617370744
:101110004807590708F076CF80910C050E94FC0320
:1011200010E01092C4041093C3041A151B0409F0B4
:1011300050C090E080E08A159B05A0F589819A81D6
:10114000DC01ED91FC910284F385E02D0995F40119
:10115000808381E090E0EFCFE5EEE093BC00A1CF8B
:1011600080910D0590910E05A0910F05B09110058D
:10117000892B8A2B8B2B09F498CF0E945601209142
:101180000D0530910E0540910F0550911005641921
:10119000750986099709261737074807590708F080
:1011A00084CFBACFCD2809F41FCF8F2DDF91CF91F7
:1011B0001F910F91FF90EF90DF90CF90BF90AF9075
:1011C0009F908F907F906F905F904F903F902F9067
:1011D0000895F12CEACF4F925F926F927F92BF9267
:1011E000CF92DF92EF92FF920F931F93CF93DF93F3
:1011F0001F92CDB7DEB78C01B62EBA0190E080E029
:101200000E9424176B017C018EEF8983AE014F5F32
:101210005F4FBA01F801838194810E94C007698100
:1012200070E06F5F7F4F90E080E00E94241720E025
:1012300034E244E759E40E94DB172B013C01F8013A
:1012400065817681878190850E9424179B01AC017E
:10125000C301B2010E9483169B01AC01C701B60114
:101260000E9483160E94F516AB016B2DC8010E94E7
:1012700073070F90DF91CF911F910F91FF90EF9027
:10128000DF90CF90BF907F906F905F904F900895C8
:10129000CF93DF9300D0CDB7DEB769834A83FC01DB
:1012A00083819481FC01248135812230310590F0C5
:1012B000208131E0309311052093330510921205FF
:1012C0001092340521E042E050E0BE016F5F7F4F95
:1012D0000E940D050F900F90DF91CF9108958F928E
:1012E0009F92AF92BF92CF92DF92EF92FF920F93B5
:1012F0001F93CF93DF931F92CDB7DEB78C014A01C6
:101300005B0120E030E040E85FE3CB01B4010E94E4
:101310007E1687FD88C020E030EC4AE555E4C50123
:10132000B4010E94D61718163CF4812C30EC932E91
:101330003AE5A32E35E4B32EF801658176818781E5
:1013400090850E9424176B017C0120E030E040E88A
:1013500055E4C501B4010E94DB179B01AC01C70134
:10136000B6010E94831620E030E040E05FE30E9477
:10137000121620E030E040E85FE30E9411164B01B6
:101380005C0120E030E040E450E40E947E1687FDDE
:1013900051C020E030E04FE753E4C501B4010E94A2
:1013A000D617181634F4812C912C9FE7A92E93E4BC
:1013B000B92E1982AE014F5F5F4FBA01F8018381E8
:1013C00094810E94C007F9804F2D4F76406160E004
:1013D000C8010E944809C501B4010E94F516462FB4
:1013E0006EEFC8010E9448094F2D60E0C8010E94BD
:1013F000480965E070E080E090E00E947B014F2D9D
:10140000406A60E0C8010E9448090F90DF91CF91C7
:101410001F910F91FF90EF90DF90CF90BF90AF9012
:101420009F908F900895812C912C20E8A22E2FE37D
:10143000B22E82CF812C912C80E4A82EBA2CB9CF69
:101440000F931F93CF93DF93EC018B819C810097C7
:1014500011F00E94451986E090E00E94A9188C01C5
:1014600089819A812881F801208392838183138264
:1014700080E290E0958384831C830B830E94E503C4
:1014800081E0F8018383C8010E942B05182F88236F
:10149000D1F040E860E0CE010E9448096AE070E0C7
:1014A00080E090E00E947B0180E498E7ADE7B1E046
:1014B0008D839E83AF83B88740E050E06AE774E491
:1014C000CE010E946F09812FDF91CF911F910F9163
:1014D0000895CF92DF92EF92FF921F93CF93DF9305
:1014E000809176028295807F80930201C091B4043E
:1014F000D091B504209769F0CE010E948A038DE057
:1015000091E099838883CE010E948A03CE010E94D4
:1015100045198FE190E00E94A918EC01F090750246
:10152000109174021B821A8288EE93E0A0E0B0E072
:101530008C839D83AE83BF838DE091E09983888304
:101540001F8A1E8A198E188E1B8E1A8E1D8E1C8E57
:101550006E8D6E7F6D7F6E8F6695617081E06827FE
:101560008F2D0E940A018F2D90E0AC014E565E4FE8
:10157000FA01649182589E4FFC012491222399F034
:1015800030E0220F331FF901EE58FF4FA591B491BF
:10159000F901EC58FE4F259134912FB7F8943C9106
:1015A000632B6C932FBFFA014491488BFC0184910B
:1015B000E82FF0E0EE0FFF1FEC58FE4F859194915D
:1015C0009A8B898B812F90E09C012E563E4F6901AA
:1015D000F9012491AC0142585E4F7A01FA018491DD
:1015E0008823C9F090E0880F991FFC01EE58FF4F47
:1015F000A591B491FC01EC58FE4F459154913FB731
:10160000F8949C91822F809598239C93FA01908165
:10161000892380833FBF8E8D81FD04C061E0812FCF
:101620000E940A011C87F601C490CD86F701E49060
:10163000EE2DF0E0EE0FFF1FE859FF4F85919491DA
:101640009F878E87D093B504C093B4042091700215
:101650003091710240917202509173021B8E1A8E6A
:10166000198E188E1F8A1E8A60E079E08DE390E063
:101670000E946A18B901C90103972430310510F49A
:1016800081E090E09D8F8C8F163108F055C0C90124
:10169000969587958431910508F491C043979F8B67
:1016A0008E8BC90105976630710510F481E090E0DA
:1016B000998F888FC901880F991F280F391F369578
:1016C0002795369527952D30310508F47BC02C5091
:1016D00031093B8F2A8F9091680084E0183048F0E0
:1016E00021E01E3008F420E081E001C0880F2A9537
:1016F000EAF7892B809368009C852DE630E09830CE
:1017000050F02BE630E09E3030F02CE630E09631A1
:1017100010F030E020E03C8B2B8B292F30E098300C
:1017200008F053C081E001C0880F9A95EAF78D8BCD
:101730008C8D9D8D0197F1F78A8D9B8D892BE1F022
:101740008091CC019091CD01C817D907A9F00097DD
:1017500011F00E948A038E8D8E7F8E8F1092CA01A7
:101760001092CB01D093CD01C093CC01EB89FC89C1
:1017700080819D89892B808380917602823090F1CF
:101780008EED95E00E94200A80EC9CEFABE9B1E081
:101790008093E3059093E405A093E505B093E605F7
:1017A00040E050E068E472E48EED95E0DF91CF9187
:1017B0001F91FF90EF90DF90CF900C946F0981E024
:1017C00090E06DCF21E030E084CF9E3040F428508F
:1017D000310981E001C0880F2A95EAF7A8CF2E5081
:1017E0003109F7CFDF91CF911F91FF90EF90DF90FC
:1017F000CF900895FB0101900020E9F73197AF01E8
:10180000461B570BDC01ED91FC910280F381E02D2A
:1018100009940F931F93CF93DF93EC010E94AD01C6
:101820008C016FE371E0CE010E94FA0B800F911FD3
:10183000DF91CF911F910F91089585ED8093BC00AA
:1018400080910D0590910E05A0910F05B0911005A6
:101850000796A11DB11D23E0B695A795979587958D
:101860002A95D1F72091BC0024FD03C010920B05EE
:10187000089540910D0550910E0560910F057091EE
:101880001005452B462B472B69F30097A105B105A1
:1018900041F02AE22A95F1F700C00197A109B109A8
:1018A000E1CF80910C050C94FC034F925F926F92F4
:1018B0007F928F929F92AF92BF92CF92DF92EF92E0
:1018C000FF920F931F93CF93DF93CDB7DEB76E9741
:1018D0000FB6F894DEBF0FBECDBFFC015C0182E6FF
:1018E000A80EB11CD5018C9194962D018823A1F0EE
:1018F000CD90DD90ED90FC90380149016C187D0889
:101900008E089F087401630185E6C816D104E104BE
:10191000F10410F0D5011C92D2010D931D932D936B
:101920003C931397D5019C91923009F46CC27A01D3
:101930008F01933040F4992359F1913009F45CC23E
:10194000F501108238C0933009F46DC29430C1F7AC
:10195000EB59FF4F80818613F3CFF12C6801F3E63A
:10196000CF0ED11CD6018C91F81650F7F801EF0D6F
:10197000F11DEA59FF4F60816F3F41F080910201F4
:10198000F81620F470E08F2D0E94D805F394EACF6A
:1019900081E06F3F09F460C26A3009F00EC2EF596E
:1019A000FF4FD080C801805A9F4F5C01DD20D1F0ED
:1019B0001082D5011C926E960FB6F894DEBF0FBE52
:1019C000CDBFDF91CF911F910F91FF90EF90DF90EE
:1019D000CF90BF90AF909F908F907F906F905F90CF
:1019E0004F900895DC01EC91EE2319F3E00FF12FF5
:1019F000F11D1082C80101969E8F8D8FD801EC9148
:101A0000EF53E83108F026C00E2E000CFF0BE55F07
:101A1000F24F0C948918C50E2A0D2A0D2A0D340D8B
:101A20002A0D2A0D2A0D2A0D3A0D2A0D2A0DE00D38
:101A3000300D230D2A0D2A0D2A0D2A0D600D880D5B
:101A40002A0D370DC40D47ED56E061E00E94A81144
:101A50008111AFCF60E970E0C7010E94090CA9CFE6
:101A60004EE956E062E0F2CF4CE856E0EECF4CE5AE
:101A700056E0F8CFF80181818111ECCF809102010D
:101A8000D81608F096CFED2DF0E0809142019091AC
:101A90004301A0914401B09145010D2C04C0B695BD
:101AA000A795979587950A94D2F780FF07C0E253D0
:101AB000FE4F608170E08D2D0E94D805D394DECF5B
:101AC00011968C918111C6CF80910201D816B8F47D
:101AD0008091980390919903A0919A03B0919B03F0
:101AE0000D2C04C0B695A795979587950A94D2F7C3
:101AF00080FF03C08D2D0E94AA07D394E5CF1092DA
:101B000098031092990310929A0310929B0351CF5D
:101B1000F801818181119ECFD090020140909803FD
:101B20005090990360909A0370909B0328EFE22EE7
:101B300022E0F22E10E000E00D1508F03ACFD301BC
:101B4000C201002E04C0B695A795979587950A9473
:101B5000D2F780FF13C0C80188589C4F4C0120E089
:101B600030E040E05FE3D7016D917D918D919C91D4
:101B70000E9412160E94F516F40160830F5F1F4F3A
:101B8000F4E0EF0EF11CD8CFCE014D960E946F11FC
:101B900097FD60CFED8DFE8D208121115BCFDC01A3
:101BA000CB01803127E29207A105B10524F08FE037
:101BB00097E2A0E0B0E09093010180930001F9CE9C
:101BC00011962C9121113EC06CE770E0CA010E9471
:101BD000AD0140917002509171026091720270915A
:101BE00073022AE0C7010E943A1260E2C7010E9414
:101BF00068114091740250E070E060E02AE0C70193
:101C00000E943A1260E2C7010E9468114091750279
:101C100050E070E060E02AE0C7010E943A1260E202
:101C2000C7010E9468114091760250E070E060E0C8
:101C30002AE0C7010E943A126FE371E0C7010E94D7
:101C4000FA0BB7CE9C8F8B8F8E010F5F1F4FCE018B
:101C50004B960E946F11F801619371938193919358
:101C60008F0197FDF7CEF3E0DF1649F0EB8DFC8D89
:101C700080818A3309F0EECE3196FC8FEB8FD394BE
:101C800094E0692ED610E3CFEB8DFC8D808181111D
:101C9000E1CE8D859E85AF85B8898F3F9105A105E1
:101CA000B10529F024F08FEF90E0A0E0B0E0982F8C
:101CB00049855A856B857C854F3F510561057105C6
:101CC00029F024F04FEF50E060E070E00D811E81BC
:101CD0002F8138850F3F11052105310529F024F0AA
:101CE0000FEF10E020E030E0E9818E2F6A815B8108
:101CF0007C81E3E4F2E5FA8BE98B8B8B6C8B5D8B5B
:101D00007E8B0F8B488F998F75EA872789278427C9
:101D10008027862785278A8FCE0141960E94420719
:101D200067E870E0882309F497CE8AE0FE01719697
:101D3000AEE6B2E001900D928A95E1F78EE6C82EEC
:101D400082E0D82E10E000E0D6019D906D01C80120
:101D50000E94FB15981621F0692DC8010E940316F8
:101D60000F5F1F4F0A30110579F762E870E0C70175
:101D70000E94090CD701ED91FC910680F781E02DBE
:101D8000C70109950E94690A14CEF8018181811169
:101D900061CE6BE870E0CA010E94AD012AE041E02B
:101DA00050E060E070E0C7010E943A1260E2C701B3
:101DB0000E946811409102012BCF6D3009F4FBCDD8
:101DC000DF01AF59BF4F8C918111F5CDE05AFF4F24
:101DD00080818F3540F491E0980F9083080F111D9A
:101DE000F8016083E8CD81E08C93108260E970E0B7
:101DF000CA010E94090CDFCD82E06E3F09F080E04D
:101E0000D5018C93D8CD8FEF860F803208F098CD16
:101E1000DF01AD59BF4F6C9311961C92EB59FF4FE8
:101E2000108283E0EDCFDF01AC59BF4FEC9191E020
:101E30009E0F9C93E00FF12FF11DEA59FF4F608335
:101E4000F801EB59FF4F8081680F608332978081E2
:101E5000981708F4B0CD84E0F5018083ACCD1F92D3
:101E60000F920FB60F9211242F933F938F939F934E
:101E7000AF93BF938091B7049091B804A091B90437
:101E8000B091BA043091B60423E0230F2D3758F5F2
:101E90000196A11DB11D2093B6048093B7049093C1
:101EA000B804A093B904B093BA048091BB04909194
:101EB000BC04A091BD04B091BE040196A11DB11D4A
:101EC0008093BB049093BC04A093BD04B093BE0464
:101ED000BF91AF919F918F913F912F910F900FBE26
:101EE0000F901F90189526E8230F0296A11DB11D93
:101EF000D2CF1F920F920FB60F9211242F933F93C0
:101F00004F935F936F937F938F939F93AF93BF9301
:101F1000EF93FF9385E395E00E944F02FF91EF91CD
:101F2000BF91AF919F918F917F916F915F914F91F1
:101F30003F912F910F900FBE0F901F9018951F92F9
:101F40000F920FB60F9211242F938F939F93EF93BD
:101F5000FF93E0914505F09146058081E0914B05A6
:101F6000F0914C0582FD1BC0908180914E058F5FE2
:101F70008F7320914F05821741F0E0914E05F0E0FC
:101F8000EB5CFA4F958F80934E05FF91EF919F91F7
:101F90008F912F910F900FBE0F901F9018958081F9
:101FA000F4CF1F920F920FB60F9211242F933F93ED
:101FB0004F935F936F937F938F939F93AF93BF9351
:101FC000EF93FF93E091CC01F091CD01309749F070
:101FD000A685B7858585968D91FF14C09C91892330
:101FE000A1F4FF91EF91BF91AF919F918F917F915C
:101FF0006F915F914F913F912F910F900FBE0F9076
:102000001F9018959C91892361F7A389B4899C91AD
:102010008589809589238C93868997890197F1F723
:10202000608D718DA685B785558538E020E0CB01A0
:102030000197F1F7822F90E095958795282F4C9185
:10204000452309F02068315091F7868D81FD209558
:102050008091CA0190E001968F7399273091CB014E
:10206000381799F0A091CA01B0E0A657BE4F2C9343
:102070008093CA01828D938D0197F1F7A389B4896A
:102080008C919589892B8C93ACCF868D8160868FBE
:10209000F1CF1F920F920FB60F9211242F933F93FF
:1020A0004F935F936F937F938F939F93AF93BF9360
:1020B000EF93FF938091B900887F803609F44AC07E
:1020C000F0F5883209F4A7C018F5803109F49BC0F7
:1020D000B8F4882309F4F9C0883009F494C0FF915A
:1020E000EF91BF91AF919F918F917F916F915F9190
:1020F0004F913F912F910F900FBE0F901F90189509
:10210000883109F488C0803251F78093090514C0E2
:10211000803409F49DC040F48033B9F38833F9F674
:102120008093090585ECB0C0803509F485C08835F9
:1021300009F496C0883499F60E941D0CD0CF8839D6
:1021400009F48CC038F5883729F050F4883611F03E
:10215000803729F683E080930B051092890157C0E0
:10216000883809F47BC0803919F0803809F0B7CF7E
:1021700080918901803208F071C0E091890181E08D
:102180008E0F809389018091BB00F0E0E759FE4FEC
:1021900080833DC0803B39F0E0F4803A09F479C097
:1021A000883A09F09CCF84E080930B051092680177
:1021B00010926701E091C104F091C20409958091E9
:1021C000670181110FC081E0809367011092470180
:1021D00009C0803C09F4A6CF883C09F4A3CF883B12
:1021E00009F07DCFE091680181E08E0F8093680156
:1021F000F0E0E95BFE4F80818093BB009091680125
:102200008091670129C08091E6048093BB0085EC32
:102210008093BC0064CF90910805809107059817C2
:1022200058F5E091080581E08E0F80930805F0E0F5
:10223000E951FB4F8081E9CFE091080581E08E0FE5
:10224000809308058091BB00F0E0E951FB4F80834B
:1022500090910805809107059817C8F285E8D8CFB6
:10226000E091080581E08E0F809308058091BB0006
:10227000F0E0E951FB4F808380910A0581115CCF2A
:1022800081E08093E50484EA8093BC0010920B0502
:1022900026CF85EC8093BC0010920B0580918901BC
:1022A000803230F4E0918901F0E0E759FE4F10826E
:1022B0006091890170E0E091BF04F091C00489E66B
:1022C00091E00995109289010ACF1092090534CF47
:1022D000DC01ED91FC910190F081E02D09941F93B8
:1022E000CF93DF93EC01E881F981808180538A30BC
:1022F00030F520E030E0A901E881F981108180ED1E
:10230000810F8A30F8F4AAE0B0E00E948F18212FE4
:10231000110F330B20533109032E000C440B550BC6
:10232000260F371F481F591F203886E9380788E9CC
:102330004807510524F43196F983E883DDCF2FEF68
:102340003FEFA901CA01B901DF91CF911F91089513
:102350007F928F929F92AF92BF92CF92DF92EF9235
:10236000FF920F931F93CF93DF9300D0CDB7DEB7CB
:102370009A838983FC0180818A01762E811113C0A2
:1023800080E00F900F90DF91CF911F910F91FF9000
:10239000EF90DF90CF90BF90AF909F908F907F9005
:1023A00008958111EDCFE981FA818081882309F4B4
:1023B0005FC0CE0101960E946F116B017C01F7FC9A
:1023C000DFCFE981FA8180818A33D1F63196FA83B1
:1023D000E983CE0101960E946F114B015C01B7FCAD
:1023E000CFCFF2E060E070E0CB017F1216C0E98150
:1023F000FA8180818A3321F63196FA83E983CE010E
:1024000001960E946F1197FDBBCF40E355E7613302
:1024100025E77207810591050CF4AB0181E388166D
:1024200085E79806A104B10434F080E3882E85E79F
:10243000982EA12CB12CD701C6018F3F9105A10583
:10244000B10529F024F08FEF90E0A0E0B0E0B401F6
:10245000F8010995E981FA8180818C3209F0A1CFD8
:10246000CF0101969A838983818181119CCF88CF86
:1024700081E087CF8F929F92AF92BF92EF92FF92AF
:102480000F931F93CF93DF93CDB7DEB7A1970FB60E
:10249000F894DEBF0FBECDBF7C01FA01CB0119A2BB
:1024A000223008F42AE08E010F5D1F4F822E912CFE
:1024B000B12CA12CBF01A50194010E944818F9017B
:1024C000CA016A300CF5605DD8016E938D01232B33
:1024D000242B252B79F790E080E0109721F0BD01A7
:1024E000C7010E94FA0BA1960FB6F894DEBF0FBE8B
:1024F000CDBFDF91CF911F910F91FF90EF90BF90D3
:10250000AF909F908F900895695CDECFE5E3F5E092
:102510001382128288EE93E0A0E0B0E0848395837A
:10252000A683B7832FE131E03183208325EC30E0AF
:102530003587248724EC30E03787268720EC30E08D
:10254000318B208B21EC30E0338B228B22EC30E07E
:10255000358B248B26EC30E0378B268B118E128E38
:10256000138E148EE2EDF5E013821282848395833C
:10257000A683B78381E391E091838083A7EEB5E0E2
:1025800080E48C931296FC93EE93119714961C9210
:102590001E921397AEEDB5E081E48C931296FC93F6
:1025A000EE93119714961C921E9213970895CF9351
:1025B000DF93CDB7DEB72E970FB6F894DEBF0FBE10
:1025C000CDBF789484B5826084BD84B5816084BDBC
:1025D00085B5826085BD85B5816085BD80916E00C1
:1025E000816080936E0010928100809181008260F2
:1025F000809381008091810081608093810080912F
:1026000080008160809380008091B100846080931D
:10261000B1008091B00081608093B00080917A0019
:10262000846080937A0080917A00826080937A003F
:1026300080917A00816080937A0080917A0080682E
:1026400080937A001092C1000EE612E01A8219827D
:1026500089819A810E94FB15D8018D938D01E981B2
:10266000FA813196FA83E9833A9791F78EE692E000
:102670000E94420781111DC083E492E590936F028E
:1026800080936E0280E895E2A0E0B0E08093700253
:1026900090937102A0937202B09373028AE08093C8
:1026A00074028BE08093750281E080937602109231
:1026B0007702C0907002D0907102E0907202F090A8
:1026C000730260E079E08DE390E0A70196010E943B
:1026D00048182150310941095109569547953795B8
:1026E0002795E0914505F091460582E08083C1146D
:1026F000F1EEDF06E104F10421F0211540E1340799
:10270000A8F0E0914505F0914605108260E874E874
:102710008EE190E0A70196010E94481821503109EE
:10272000410951095695479537952795E0914105FF
:10273000F09142053083E0914305F09144052083F8
:1027400010924D05E0914905F0914A0586E080839D
:10275000E0914705F0914805808180618083E09198
:102760004705F0914805808188608083E0914705A6
:10277000F0914805808180688083E0914705F09161
:10278000480580818F7D80830E94E50387EE95E078
:102790000E94200A80EC9CEFABE9B1E08093EC054D
:1027A0009093ED05A093EE05B093EF0540E050E067
:1027B00068E472E487EE95E00E946F092EE2822EB3
:1027C00022E0922E8EEE91E09C878B8734EDC32E13
:1027D00030E0D32E4EEC642E41E0742E54EBE52E07
:1027E00050E0F52E68ED462E62E0562E04E910E02A
:1027F00078EB272E72E0372EA8EFB2E0B887AF83D0
:10280000E8E7F3E0FA83E98328E732E03C832B83AF
:102810001E861D86ED85FE85EC5CFE4F85919491AC
:10282000D4018D939D934D01ED85FE85EC50FF4FB6
:1028300085919491EB85FC8581939193FC87EB873F
:10284000F601B490D301BD923D01F7018491D2010C
:102850008D932D01F8018491D1018D931D016B2D74
:1028600070E090E080E00E942417EF81F88561938A
:10287000719381939193F887EF83A981BA81BD9277
:10288000BA83A983EB81FC8111921192FC83EB83C3
:10289000FFEFCF1ADF0A2FEFE21AF20A0F5F1F4F86
:1028A0004D855E854E5F5F4F5E874D874034510595
:1028B00009F0B0CF0E94690A198280910201598102
:1028C000581738F4852F0E94AA0789818F5F898362
:1028D000F4CF8AE8EAE2F4E0DF01282F1D922A957E
:1028E000E9F7E0EAF3E0DF011D928A95E9F72FB7F7
:1028F000F8948091B7049091B804A091B904B09174
:10290000BA042FBF80939C0390939D03A0939E03D2
:10291000B0939F038091B4049091B504DC01ED91D4
:10292000FC910084F185E02D0995892B21F18FB769
:10293000F894C090B704D090B804E090B904F09037
:10294000BA048FBFE091B404F091B504FA83E9832F
:102950000190F081E02D0284F385E02D89819A8138
:1029600009959701860149815A81682F8AE294E08E
:102970000E94550CCFCF85E395E00E942F02892B52
:10298000C9F08FB7F894C090B704D090B804E09025
:10299000B904F090BA048FBF85E395E00E940D0260
:1029A0009701860145E355E0682F80EA93E00E9495
:1029B000550CE1CF8FB7F894C090B704D090B8040D
:1029C000E090B904F090BA048FBF80919C0390917D
:1029D0009D03A0919E03B0919F03A7019601281B20
:1029E000390B4A0B5B0BCA01B901643171058105D2
:1029F000910508F4F3C00E94241720E030E04AE774
:102A000054E40E9483166F83788789879A87C092DF
:102A10009C03D0929D03E0929E03F0929F0310E0EE
:102A200080910201181708F0D9C0212E312C809115
:102A3000980390919903A0919A03B0919B03012E62
:102A400004C0B695A795979587950A94D2F780FF0D
:102A5000A5C0F101E858FC4F608170E090E080E093
:102A60000E9424172B013C01E0900001F09001012D
:102A7000A101440F551F440F551F5A834983FA0182
:102A8000E850FD4FE114F10409F4A3C089819A8153
:102A900088509D4F9C878B87DC018D909D90AD90D9
:102AA000BC90A5019401C301B2010E9411166B8371
:102AB0007C838D839E83B70190E080E00E94241781
:102AC0002F81388549855A850E94DB176B017C016F
:102AD000AC019B016B817C818D819E810E94D61708
:102AE000A701960118160CF05BC0C501B4010E9445
:102AF0001216EB85FC856083718382839383E98161
:102B0000FA81E850FD4F4081518162817381812FAC
:102B10000E94DE06F82E092FF101E852FD4F608178
:102B200070E090E080E00E942417AB01BC01812F8F
:102B30000E94DE069A838983F101E854FD4F60818B
:102B400070E090E080E00E942417AB01BC01812F6F
:102B50000E94DE062F2D302F49815A812417350718
:102B600008F49A01AC012817390708F4A901F1010A
:102B7000EE0FFF1FE858FD4F8081918148175907DC
:102B800069F05183408360EF610F8EED95E0103165
:102B900018F4612F87EE95E00E94EB081F5F40CF8D
:102BA00050586B817C818D819E810E947E1687FFAB
:102BB0000EC0A7019601C501B4010E941116AB8594
:102BC000BC856D937D938D939C93139798CFEB85E4
:102BD000FC85408251826282738291CF80E090E0D6
:102BE000892B09F497CE0E943B02882309F492CEE8
:102BF0000E9400008FCEF999FECF92BD81BDF89A58
:102C0000992780B50895262FF999FECF1FBA92BD56
:102C100081BD20BD0FB6F894FA9AF99A0FBE0196BD
:102C200008955058BB27AA270E9429160C949C1778
:102C30000E948E1738F00E94951720F039F49F3FBC
:102C400019F426F40C948B170EF4E095E7FB0C9422
:102C50008517E92F0E94AD1758F3BA17620773075B
:102C60008407950720F079F4A6F50C94CF170EF49D
:102C7000E0950B2EBA2FA02D0B01B90190010C018C
:102C8000CA01A0011124FF27591B99F0593F50F4A4
:102C9000503E68F11A16F040A22F232F342F4427FC
:102CA000585FF3CF469537952795A795F0405395F4
:102CB000C9F77EF41F16BA0B620B730B840BBAF0C4
:102CC0009150A1F0FF0FBB1F661F771F881FC2F72F
:102CD0000EC0BA0F621F731F841F48F48795779543
:102CE0006795B795F7959E3F08F0B0CF9395880FFD
:102CF00008F09927EE0F9795879508950E94611720
:102D000008F481E008950E9497160C949C170E9485
:102D1000951758F00E948E1740F029F45F3F29F074
:102D20000C94851751110C94D0170C948B170E949A
:102D3000AD1768F39923B1F3552391F3951B550B08
:102D4000BB27AA2762177307840738F09F5F5F4F7E
:102D5000220F331F441FAA1FA9F335D00E2E3AF0BD
:102D6000E0E832D091505040E695001CCAF72BD0D5
:102D7000FE2F29D0660F771F881FBB1F2617370726
:102D80004807AB07B0E809F0BB0B802DBF01FF2758
:102D900093585F4F3AF09E3F510578F00C94851799
:102DA0000C94D0175F3FE4F3983ED4F38695779563
:102DB0006795B795F7959F5FC9F7880F911D969511
:102DC000879597F90895E1E0660F771F881FBB1F6D
:102DD000621773078407BA0720F0621B730B840B1A
:102DE000BA0BEE1F88F7E09508950E94B51788F09A
:102DF0009F5798F0B92F9927B751B0F0E1F0660FBF
:102E0000771F881F991F1AF0BA95C9F714C0B130FF
:102E100091F00E94CF17B1E008950C94CF17672F5F
:102E2000782F8827B85F39F0B93FCCF3869577952E
:102E30006795B395D9F73EF4909580957095619517
:102E40007F4F8F4F9F4F0895E89409C097FB3EF442
:102E500090958095709561957F4F8F4F9F4F9923E7
:102E6000A9F0F92F96E9BB279395F6958795779565
:102E70006795B795F111F8CFFAF4BB0F11F460FF25
:102E80001BC06F5F7F4F8F4F9F4F16C0882311F07D
:102E900096E911C0772321F09EE8872F762F05C091
:102EA000662371F096E8862F70E060E02AF09A952C
:102EB000660F771F881FDAF7880F9695879597F921
:102EC0000895990F0008550FAA0BE0E8FEEF1616BB
:102ED0001706E807F907C0F012161306E407F5070E
:102EE00098F0621B730B840B950B39F40A2661F082
:102EF000232B242B252B21F408950A2609F4A14025
:102F0000A6958FEF811D811D089597F99F6780E831
:102F100070E060E008959FEF80EC089500240A942B
:102F20001616170618060906089500240A941216A4
:102F30001306140605060895092E0394000C11F4D7
:102F4000882352F0BB0F40F4BF2B11F460FF04C084
:102F50006F5F7F4F8F4F9F4F089557FD9058440FDD
:102F6000551F59F05F3F71F04795880F97FB991FE8
:102F700061F09F3F79F087950895121613061406A5
:102F8000551FF2CF4695F1DF08C016161706180632
:102F9000991FF1CF86957105610508940895E8940D
:102FA000BB2766277727CB0197F908950E94611701
:102FB00008F48FEF08950E94EE170C949C170E945E
:102FC0008E1738F00E94951720F0952311F00C947D
:102FD00085170C948B1711240C94D0170E94AD17F1
:102FE00070F3959FC1F3950F50E0551F629FF0015C
:102FF000729FBB27F00DB11D639FAA27F00DB11D75
:10300000AA1F649F6627B00DA11D661F829F2227FD
:10301000B00DA11D621F739FB00DA11D621F839F84
:10302000A00D611D221F749F3327A00D611D231F5A
:10303000849F600D211D822F762F6A2F11249F57A8
:1030400050409AF0F1F088234AF0EE0FFF1FBB1FAB
:10305000661F771F881F91505040A9F79E3F51056A
:1030600080F00C9485170C94D0175F3FE4F3983EE2
:10307000D4F3869577956795B795F795E7959F5F14
:10308000C1F7FE2B880F911D9695879597F90895A6
:10309000A1E21A2EAA1BBB1BFD010DC0AA1FBB1F5C
:1030A000EE1FFF1FA217B307E407F50720F0A21BCE
:1030B000B30BE40BF50B661F771F881F991F1A943B
:1030C00069F760957095809590959B01AC01BD0165
:1030D000CF010895052E97FB1EF400940E948118DD
:1030E00057FD07D00E94481807FC03D04EF40C94FB
:1030F000811850954095309521953F4F4F4F5F4F28
:10310000089590958095709561957F4F8F4F9F4F53
:103110000895EE0FFF1F0590F491E02D09940E9491
:103120009A18A59F900DB49F900DA49F800D911D9E
:1031300011240895A29FB001B39FC001A39F700DF9
:10314000811D1124911DB29F700D811D1124911DAF
:1031500008950F931F93CF93DF938230910510F45E
:1031600082E090E0E091F205F091F30530E020E09C
:10317000B0E0A0E0309799F42115310509F44AC078
:10318000281B390B24303105D8F58A819B816115C4
:10319000710589F1FB0193838283FE0111C0408197
:1031A00051810281138148175907E0F048175907E8
:1031B00099F4109761F012960C93129713961C9342
:1031C0003296CF01DF91CF911F910F910895009317
:1031D000F2051093F305F4CF2115310551F0421794
:1031E000530738F0A901DB019A01BD01DF01F801A5
:1031F000C1CFEF01F9CF9093F3058093F205CDCFC6
:10320000FE01E20FF31F819391932250310939831C
:103210002883D7CF2091F0053091F105232B41F47D
:1032200020910501309106013093F1052093F005BE
:1032300020910301309104012115310541F42DB78E
:103240003EB74091070150910801241B350BE091D6
:10325000F005F091F105E217F307A0F42E1B3F0BE8
:103260002817390778F0AC014E5F5F4F24173507F8
:1032700048F04E0F5F1F5093F1054093F005819386
:1032800091939FCFF0E0E0E09CCFCF93DF93009746
:10329000E9F0FC01329713821282A091F205B091FD
:1032A000F305ED0130E020E01097A1F42081318199
:1032B000820F931F2091F0053091F10528173907EF
:1032C00009F061C0F093F105E093F005DF91CF9133
:1032D0000895EA01CE17DF07E8F54A815B819E0178
:1032E00041155105B1F7E901FB83EA8349915991F1
:1032F000C40FD51FEC17FD0761F480819181029600
:10330000840F951FE90199838883828193819B8330
:103310008A83F0E0E0E012968D919C9113970097DC
:10332000B9F52D913C911197CD010296820F931F13
:103330002091F0053091F1052817390739F63097BB
:1033400051F51092F3051092F205B093F105A09398
:10335000F005BCCFD383C28340815181840F951F78
:10336000C817D90761F44E5F5F4F88819981480F74
:10337000591F518340838A819B81938382832115C6
:10338000310509F0B0CFF093F305E093F2059ECF3D
:10339000FD01DC01C0CF13821282D7CFF894FFCF9A
:1033A0007800100000F405800000000000F702D152
:1033B00001D505F60253036903DE02000000007127
:1033C00002D101FE01BE022F020D02210200000007
:1033D00000A6057905D505F60272055F0550050DB5
:0233E0000A00E1
:00000001FF
